:10000000FD28A0007F39201B803C0920A01B003C5C
:1000100008008A01820700340334063409340C34A2
:1000200010341334163419341C341F34223425345C
:1000300028342B342E3431343334363439343C3490
:100040003F3441344434473449344C344E345134D1
:100050005334553458345A345C345E34603462342A
:100060006434663468346A346B346D346F3470349D
:1000700071347334743475347634783479347A3432
:100080007A347B347C347D347D347E347E347E34EB
:100090007F347F347F347F34A4002508A402031CFE
:1000A000A5032708A602031CA7033709A2003509E8
:1000B000A300A20A0319A30A4130A900AC01AD01B3
:1000C000AE01AF01A8013608840034098E208413E4
:1000D000F9202408AC070318AD0A2508AD07260847
:1000E000AE070318AF0A2708AF072D080120803E8E
:1000F000A1002F080120803EA107210CA8070008BD
:100100003404031C34068000290303194130A9007C
:100110000319A20A0319A30F6828F8288417800579
:10012000F8289620B4000408B6000800A80005309E
:10013000A8190530840000308A0028080739820792
:100140000134023404340834103420344034803410
:100150000F39A0000310A00DA00D1F08E0392004E6
:1001600001389F000030A1003230CC209F149F182E
:10017000B7281E08A10083161E08F828A301A200B4
:10018000FF30A207031CA307031CF8280330A100BB
:10019000E630CC20C028A101FC3EA000A109031C30
:1001A000D728FF300000A0070318D228A00764005A
:1001B000A10FD1280800A2000130E128A2000630DA
:1001C000E128A80023082102031DE82822082002B4
:1001D000043003180130031902302805031DFF30D5
:1001E000F8280038031DFF300405031DFF30F828F0
:1001F0008313031383126400080089309F000230C8
:10020000A820B8002108B9000A30BE203808A00094
:100210003908A100A3012530DE20031D102911217A
:10022000FF283808A0003908A1000330A30092304D
:10023000DB20BA003808A0003908A1000330A30071
:10024000FF30DE20BC003A0884003C08F120BC00EE
:10025000BD0064003C083D0403193B290030912097
:100260007830B700B5018430A6000330A700023013
:10027000A500BC304C203808A0003908A10003308C
:10028000A3004930DB20BA003808A0003908A100DB
:100290000330A3009230DE20BC003A0884003C0802
:1002A000F120BC00BD0064003C083D040319652931
:1002B000003091207830B700B5014C30A6000430F2
:1002C000A7000230A500BC304C203808A000390837
:1002D000A1000230A300FF30DB20BA003808A000E4
:1002E0003908A1000330A3004930DE20BC003A08E1
:1002F00084003C08F120BC00BD0064003C083D04C3
:1003000003198F29003091207830B700B5014C30A7
:10031000A6000430A7000330A50084304C20380824
:10032000A0003908A1000230A300B630DB20BA00DB
:100330003808A0003908A1000230A300FF30DE20F9
:10034000BC003A0884003C08F120BC00BD006400F9
:100350003C083D040319B929003091207830B700DA
:10036000B5011430A6000530A7000230A500BC304E
:100370004C203808A0003908A1000230A3006D30DD
:10038000DB20BA003808A0003908A1000230A30021
:10039000B630DE20BC003A0884003C08F120BC00E6
:1003A000BD0064003C083D040319E329003091209E
:1003B0007830B700B5011430A6000530A70003302F
:1003C000A50084304C203808A0003908A100023074
:1003D000A3002530DB20BA003808A0003908A100AE
:1003E0000230A3006D30DE20BC003A0884003C08D7
:1003F000F120BC00BD0064003C083D0403190D2A37
:10040000003091207830B700B5011430A6000530D7
:10041000A7000430A5004C304C203808A000390853
:10042000A1000130A300DB30DB20BA003808A000B7
:100430003908A1000230A3002530DE20BC003A08B4
:1004400084003C08F120BC00BD0064003C083D0471
:100450000319372A003091207830B700B501DC301D
:10046000A6000530A7000230A500BC304C2038089B
:10047000A0003908A1000130A3009130DB20BA00B0
:100480003808A0003908A1000130A300DB30DE20CD
:10049000BC003A0884003C08F120BC00BD006400A8
:1004A0003C083D040319612A003091207830B700E0
:1004B000B501DC30A6000530A7000330A50084306C
:1004C0004C203808A0003908A1000130A3004930B1
:1004D000DB20BA003808A0003908A1000130A300D1
:1004E0009130DE20BC003A0884003C08F120BC00BA
:1004F000BD0064003C083D0403198B2A00309120A4
:100500007830B700B501DC30A6000530A700043014
:10051000A5004C304C203808A0003908A10001305B
:10052000A3000030DB20BA003808A0003908A10081
:100530000130A3004930DE20BC003A0884003C08AA
:10054000F120BC00BD0064003C083D040319B52A3D
:10055000003091207830B700B501A430A6000630F5
:10056000A7000430A5004C304C203808A000390802
:10057000A100A301B630DB20BA003808A00039087A
:10058000A1000130A3000030DE20BC003A08840046
:100590003C08F120BC00BD0064003C083D04031988
:1005A000DE2A003091207830B700B501DC30A6009B
:1005B0000530A7000530A50014304C203808A000F5
:1005C0003908A100A3016E30DB20BA003808A00072
:1005D0003908A100A301B630DE20BC003A0884002F
:1005E0003C08F120BC00BD0064003C083D04031938
:1005F000062B003091207830B700B501A430A6005A
:100600000630A7000530A500DC304C203808A000DB
:100610003908A100A3012530DB20BA003808A0006A
:100620003908A100A3016E30DE20BC003A08840026
:100630003C08F120BC00BD0064003C083D040319E7
:100640002D2B00309120E830B7000330B5000A3080
:10065000A700A5002830A6004C200230A820B80032
:100660002108B9000A30BE203808A0003908A100CE
:0C067000A3012530DB20031D2D2B08000A
:02400E00EA3096
:00000001FF
